:100000000C94460018950000189500001895000003
:10001000189500001895000018950000189500002C
:10002000189500001895000018950000189500001C
:10003000189500001895000018950000189500000C
:1000400018950000189500001895000018950000FC
:1000500018950000189500001895000018950000EC
:1000600018950000189500001895000018950000DC
:1000700018950000189500000C944F2D0C94832DBA
:100080001895000018950000189500008FEF8DBF9F
:10009000C0E8E8E94E2E80E18EBFD0E1FFE05F2EA0
:1000A000EEEFFFE0A0E0B1E0A89584B7082E877FCF
:1000B00084BF88E1992781BD91BD88278D933197B1
:1000C000E9F780E08093980080E18093990088E1CF
:1000D00080939A00662480919A00806880939A00A9
:1000E0000E948D2E8FE787BB85E08093510288E0C8
:1000F0008093520286E08093530289E080935402F9
:1001000088E0809355028EE08093560289E08093C8
:1001100057028FE0809358020E945F29709A80E016
:100120008093480280E080934D020E9482230E94C7
:10013000751881E08093480285E080934D020E940B
:100140007518ECE6FBE10E94462D0E947E285A922B
:100150004A9280E0A42DB52D8C9381E00E948F28D7
:100160005A924A9280E0A42DB52D8C9381E00E9492
:100170008F285A924A928FEAA42DB52D8C9381E054
:100180000E948F285A924A9283E8A42DB52D8C9311
:1001900081E00E948F280E948319289684E00E94A3
:1001A0008B2878940091E701013011F00C940E0136
:1001B00080E08093E7010E948D2EA7E6B1E03FE347
:1001C0000E94EA280E948A2EA9E2B1E00E94AF2D87
:1001D000A7E6B1E08C91082F0A3011F00C940C01C5
:1001E000A7E6B1E00E94702E082F41E0041BA8EEA4
:1001F000B1E00C93A7E6B1E00E94702EEA2FFB2F2E
:100200000091E8013197E01BF10B0FEFA7E6B1E099
:100210000E94682E0C94E8000E9415010C94D200F4
:1002200081E08093E70108950895A7E6B1E08C91FD
:10023000082F033211F00C941F010C949A01A7E6C9
:10024000B1E08C91082F0B3111F00C9429010C9422
:100250009A01A7E6B1E0E4E5FDE50E94462D2FEF07
:1002600091E00E94BA2AA1EFB1E00C930091F10154
:10027000003018F011F00C943F010C948C01A7E6AB
:10028000B1E0E6E5FDE50E94462D2FEF91E00E94EA
:10029000BA2A002F003080E010F009F081E08F933F
:1002A0004091F101A7E6B1E0E6E5FDE50E94462DAB
:1002B0002FEF91E00E94BA2A002F041781E008F086
:1002C00080E09F918923882311F40C946D010E9492
:1002D0009B010C949A010C948A01E7E6F1E00091ED
:1002E000F101A7EAB1E00E94682EA7EAB1E00E94FE
:1002F000242EA9EEB1E00C930091E901023011F037
:100300000C9488010E949B010C949A010C948A0120
:100310000C949A010C949A010091E901023011F0B9
:100320000C9498010E949B010C949A010C949A01E0
:100330000C949A01089581E00E948229A7E6B1E019
:100340000E94702E082F42E0041BA1EFB1E00C9335
:10035000A7E6B1E00E94702EEA2FFB2F0091F10179
:100360003197E01BF10B0FEFA7EAB1E00E94682E76
:10037000A7EAB1E0E8E5FDE50E94462D2FEF91E008
:100380000E94BA2AA1EFB1E00C930091F101003074
:1003900018F011F00C94CE010C94D30180E08093FE
:1003A000F0010C94D60181E08093F0010091F101FD
:1003B000003011F00C94E301A7EAB1E00E94702E26
:1003C000A1EFB1E08C93E7EAF1E00091F101A7E53C
:1003D000B1E00E94682EA7E5B1E00E94242EAAEEAB
:1003E000B1E00D931C930091F001003011F00C94DA
:1003F0001E02A7EAB1E00E94702E082F4091F10181
:10040000041BA0EFB1E00C93A7EAB1E00E94702EAC
:10041000EA2FFB2F0091F0013197E01BF10B0FEF5A
:10042000A7E5B1E00E94682EA7E5B1E00E940D2C7F
:10043000EDE0F0E0ACEEB1E00E945B2EAAEEB1E0A0
:100440000D911C91033050E0150711F00C948802B7
:10045000E7E5F1E0A2EFB1E013E021E001E03327AE
:100460000E94022D5A924A92E2EFF1E0A42DB52D9E
:100470000E94562E85E10E948F285A924A9288E166
:10048000A42DB52D8C9381E00E948F285A924A9218
:1004900085E5A42DB52D8C9381E00E948F285A927A
:1004A0004A9281E0A42DB52D8C9381E00E948F2883
:1004B0005A924A9281E0A42DB52D8C9381E00E943E
:1004C0008F285A924A9281E0A42DB52D8C9381E019
:1004D0000E948F285A924A9280E090E0A42DB52D78
:1004E0008D939C9382E00E948F285A924A928FEFBC
:1004F0009FEFA42DB52D8D939C9382E00E948F28B1
:100500000E94C32060968EE10E948B280C94AD0D52
:10051000073050E0150711F00C940104ECEEF1E007
:100520000E941F2BE0E2FDE50E94462D0E94EE2B6B
:100530000E94F72B10F00C94C70280E080931C02FD
:10054000E4E2FDE50E94462D0E94EE2BECEEF1E088
:100550000E941F2B0E94B42BEDE0F0E0ACEEB1E066
:100560000E945B2EE8E2FDE50E94462D0E94EE2BE4
:10057000ECEEF1E00E941F2B0E945E2BEDE0F0E01C
:100580000E94EB2AADE1B2E0DC920C94DD0280E047
:1005900080931D02E8E2FDE50E94462D0E94EE2BAD
:1005A000ECEEF1E00E941F2B0E945E2BEDE0F0E0EC
:1005B0000E94EB2AACE1B2E0DC92ECEEF1E00E94AA
:1005C0001F2BECE2FDE50E94462D0E94EE2B0E94BF
:1005D000F72B18F011F00C94EF020C94F70280E066
:1005E00098EFAEE1B2E08D939C930C94FD0280EE07
:1005F00097E0AEE1B2E08D939C9300911D0204322E
:1006000018F011F00C9406030C94090384E2809313
:100610001D020AE540911D02040FADE1B2E00C930A
:100620005A924A9284E6A42DB52D8C9381E00E94C3
:100630008F285A924A928AE5A42DB52D8C9381E099
:100640000E948F285A924A9289E6A42DB52D8C9348
:1006500081E00E948F285A924A9280911D02A42D17
:10066000B52D8C9381E00E948F285A924A92AEE178
:10067000B2E08D919C91A42DB52D8D939C9382E039
:100680000E948F280E94A81C2A9686E00E948B2830
:100690005A924A9284E6A42DB52D8C9381E00E9453
:1006A0008F285A924A9280911D02A42DB52D8C93C9
:1006B00081E00E948F285A924A9289E6A42DB52D96
:1006C0008C9381E00E948F285A924A928EE7A42D43
:1006D000B52D8C9381E00E948F285A924A928FEF19
:1006E0009FEFA42DB52D8D939C9382E00E948F28BF
:1006F0000E94A81C2A9686E00E948B2800911C026A
:10070000043218F011F00C9487030C948A0384E2ED
:1007100080931C020AE540911C02041BACE1B2E08C
:100720000C935A924A9284E6A42DB52D8C9381E0C5
:100730000E948F285A924A9280911C02A42DB52DB6
:100740008C9381E00E948F285A924A9289E6A42DC8
:10075000B52D8C9381E00E948F285A924A928AE5A7
:10076000A42DB52D8C9381E00E948F285A924A9235
:10077000AEE1B2E08D919C91A42DB52D8D939C930B
:1007800082E00E948F280E94A81C2A9686E00E9480
:100790008B285A924A9284E6A42DB52D8C9381E041
:1007A0000E948F285A924A9285E3A42DB52D8C93EE
:1007B00081E00E948F285A924A9289E6A42DB52D95
:1007C0008C9381E00E948F285A924A9280911C0259
:1007D000A42DB52D8C9381E00E948F285A924A92C5
:1007E0008FEF9FEFA42DB52D8D939C9382E00E94F7
:1007F0008F280E94A81C2A9686E00E948B280C94C1
:10080000AD0D083050E0150711F00C947D05ECEEAD
:10081000F1E00E941F2BE0E2FDE50E94462D0E94C0
:10082000EE2B0E94F72B18F011F00C9419040C9485
:10083000310480E080931D02E8E2FDE50E94462D30
:100840000E94EE2BECEEF1E00E941F2B0E945E2B2B
:10085000EDE0F0E00E94EB2AACE1B2E0DC920C9417
:10086000590480E080931C02E4E2FDE50E94462DDD
:100870000E94EE2BECEEF1E00E941F2B0E94B42BA5
:10088000EDE0F0E0ACEEB1E00E945B2EE8E2FDE5C9
:100890000E94462D0E94EE2BECEEF1E00E941F2BF1
:1008A0000E945E2BEDE0F0E00E94EB2AADE1B2E0A9
:1008B000DC92ECEEF1E00E941F2BECE2FDE50E94E1
:1008C000462D0E94EE2B0E94F72B18F011F00C948D
:1008D0006B040C94730480E098EFAEE1B2E08D936A
:1008E0009C930C94790480EE97E0AEE1B2E08D9396
:1008F0009C9300911D02043218F011F00C948204B4
:100900000C94850484E280931D020AE540911D0247
:10091000040FADE1B2E00C935A924A9286E4A42D02
:10092000B52D8C9381E00E948F285A924A928AE5D5
:10093000A42DB52D8C9381E00E948F285A924A9263
:100940008BE4A42DB52D8C9381E00E948F285A92C0
:100950004A9280911D02A42DB52D8C9381E00E94B6
:100960008F285A924A92AEE1B2E08D919C91A42DCB
:10097000B52D8D939C9382E00E948F280E94A81C25
:100980002A9686E00E948B285A924A9286E4A42DE9
:10099000B52D8C9381E00E948F285A924A928091C3
:1009A0001D02A42DB52D8C9381E00E948F285A92B0
:1009B0004A928BE4A42DB52D8C9381E00E948F2860
:1009C0005A924A928EE7A42DB52D8C9381E00E9415
:1009D0008F285A924A928FEF9FEFA42DB52D8D93B9
:1009E0009C9382E00E948F280E94A81C2A9686E091
:1009F0000E948B2800911C02043218F011F00C9414
:100A000003050C94060584E280931C020AE54091DC
:100A10001C02041BACE1B2E00C935A924A9286E4A9
:100A2000A42DB52D8C9381E00E948F285A924A9272
:100A300080911C02A42DB52D8C9381E00E948F28FB
:100A40005A924A928BE4A42DB52D8C9381E00E949A
:100A50008F285A924A928AE5A42DB52D8C9381E075
:100A60000E948F285A924A92AEE1B2E08D919C91F9
:100A7000A42DB52D8D939C9382E00E948F280E9417
:100A8000A81C2A9686E00E948B285A924A9286E4F5
:100A9000A42DB52D8C9381E00E948F285A924A9202
:100AA00085E3A42DB52D8C9381E00E948F285A9266
:100AB0004A928BE4A42DB52D8C9381E00E948F285F
:100AC0005A924A9280911C02A42DB52D8C9381E0FC
:100AD0000E948F285A924A928FEF9FEFA42DB52D36
:100AE0008D939C9382E00E948F280E94A81C2A96D6
:100AF00086E00E948B280C94AD0D093050E015075C
:100B000011F00C940407ECEEF1E00E94EB2AA4E251
:100B1000B2E0EE0C000FE794DD92EC92ECEEF1E027
:100B20000E941F2BE0E2FDE50E94462D0E94EE2B65
:100B30000E94F72B18F011F00C94A0050C94B80546
:100B400080E080931D02E8E2FDE50E94462D0E94B0
:100B5000EE2BECEEF1E00E941F2B0E945E2BEDE0ED
:100B6000F0E00E94EB2AACE1B2E0DC920C94E005EC
:100B700080E080931C02E4E2FDE50E94462D0E9485
:100B8000EE2BECEEF1E00E941F2B0E94B42BEDE067
:100B9000F0E0ACEEB1E00E945B2EE8E2FDE50E94E1
:100BA000462D0E94EE2BECEEF1E00E941F2B0E94DE
:100BB0005E2BEDE0F0E00E94EB2AADE1B2E0DC92CA
:100BC000ECEEF1E00E941F2BECE2FDE50E94462DC9
:100BD0000E94EE2B0E94F72B18F011F00C94F205F6
:100BE0000C94FA0580E098EFAEE1B2E08D939C930F
:100BF0000C9400068FE190E0AEE1B2E08D939C93FF
:100C000000911D02043218F011F00C9409060C94A6
:100C10000C0684E280931D020AE540911D02040F38
:100C2000ADE1B2E00C935A924A928BE4A42DB52D1B
:100C30008C9381E00E948F285A924A928AE5A42DD3
:100C4000B52D8C9381E00E948F285A924A9280E5BC
:100C5000A42DB52D8C9381E00E948F285A924A9240
:100C600080911D02A42DB52D8C9381E00E948F28C8
:100C70005A924A92AEE1B2E08D919C91A42DB52D8D
:100C80008D939C9382E00E948F280E94A81C2A9634
:100C900086E00E948B285A924A928BE4A42DB52DAF
:100CA0008C9381E00E948F285A924A9280911D0273
:100CB000A42DB52D8C9381E00E948F285A924A92E0
:100CC00080E5A42DB52D8C9381E00E948F285A9247
:100CD0004A928EE7A42DB52D8C9381E00E948F2837
:100CE0005A924A928FEF9FEFA42DB52D8D939C932E
:100CF00082E00E948F280E94A81C2A9686E00E940B
:100D00008B2800911C02043218F011F00C948A0612
:100D10000C948D0684E280931C020AE540911C022B
:100D2000041BACE1B2E00C935A924A928BE4A42DDE
:100D3000B52D8C9381E00E948F285A924A9280911F
:100D40001C02A42DB52D8C9381E00E948F285A920D
:100D50004A9280E5A42DB52D8C9381E00E948F28C6
:100D60005A924A928AE5A42DB52D8C9381E00E9477
:100D70008F285A924A92AEE1B2E08D919C91A42DB7
:100D8000B52D8D939C9382E00E948F280E94A81C11
:100D90002A9686E00E948B285A924A928BE4A42DD0
:100DA000B52D8C9381E00E948F285A924A9285E358
:100DB000A42DB52D8C9381E00E948F285A924A92DF
:100DC00080E5A42DB52D8C9381E00E948F285A9246
:100DD0004A9280911C02A42DB52D8C9381E00E9433
:100DE0008F285A924A928FEF9FEFA42DB52D8D93A5
:100DF0009C9382E00E948F280E94A81C2A9686E07D
:100E00000E948B280C94AD0D0A3050E0150711F0AC
:100E10000C948808ECEEF1E00E94EB2AA6E2B2E026
:100E2000EE0C000FE794DD92EC92ECEEF1E00E9404
:100E30001F2BE0E2FDE50E94462D0E94EE2B0E9452
:100E4000F72B10F00C944E0780E080931C02E4E234
:100E5000FDE50E94462D0E94EE2BECEEF1E00E9493
:100E60001F2B0E94B42BEDE0F0E0ACEEB1E00E944D
:100E70005B2EE8E2FDE50E94462D0E94EE2BECEE93
:100E8000F1E00E941F2B0E945E2BEDE0F0E00E943B
:100E9000EB2AADE1B2E0DC920C94640780E0809331
:100EA0001D02E8E2FDE50E94462D0E94EE2BECEECD
:100EB000F1E00E941F2B0E945E2BEDE0F0E00E940B
:100EC000EB2AACE1B2E0DC92ECEEF1E00E941F2BE9
:100ED000ECE2FDE50E94462D0E94EE2B0E94F72BCE
:100EE00018F011F00C9476070C947E0780E098EFD0
:100EF000AEE1B2E08D939C930C9484078FE190E077
:100F0000AEE1B2E08D939C9300911D02043218F083
:100F100011F00C948D070C94900784E280931D02CD
:100F20000AE540911D02040FADE1B2E00C935A9224
:100F30004A928FE5A42DB52D8C9381E00E948F28D5
:100F40005A924A928AE5A42DB52D8C9381E00E9495
:100F50008F285A924A9284E6A42DB52D8C9381E075
:100F60000E948F285A924A9280911D02A42DB52D7D
:100F70008C9381E00E948F285A924A92AEE1B2E0AF
:100F80008D919C91A42DB52D8D939C9382E00E9410
:100F90008F280E94A81C2A9686E00E948B285A92CD
:100FA0004A928FE5A42DB52D8C9381E00E948F2865
:100FB0005A924A9280911D02A42DB52D8C9381E006
:100FC0000E948F285A924A9284E6A42DB52D8C93C4
:100FD00081E00E948F285A924A928EE7A42DB52D67
:100FE0008C9381E00E948F285A924A928FEF9FEF54
:100FF000A42DB52D8D939C9382E00E948F280E9492
:10100000A81C2A9686E00E948B2800911C020432BC
:1010100018F011F00C940E080C94110884E28093DF
:101020001C020AE540911C02041BACE1B2E00C93E7
:101030005A924A928FE5A42DB52D8C9381E00E949F
:101040008F285A924A9280911C02A42DB52D8C9320
:1010500081E00E948F285A924A9284E6A42DB52DF1
:101060008C9381E00E948F285A924A928AE5A42D9F
:10107000B52D8C9381E00E948F285A924A92AEE15E
:10108000B2E08D919C91A42DB52D8D939C9382E01F
:101090000E948F280E94A81C2A9686E00E948B2816
:1010A0005A924A928FE5A42DB52D8C9381E00E942F
:1010B0008F285A924A9285E3A42DB52D8C9381E016
:1010C0000E948F285A924A9284E6A42DB52D8C93C3
:1010D00081E00E948F285A924A9280911C02A42D8E
:1010E000B52D8C9381E00E948F285A924A928FEFFF
:1010F0009FEFA42DB52D8D939C9382E00E948F28A5
:101100000E94A81C2A9686E00E948B280C94AD0DA4
:101110000B3050E0150711F00C945D0BE7E0F2E0A6
:10112000A7E5B1E00E94782E11F40C945B0BE7E583
:10113000F1E0A7E0B2E00E94562E5A924A92A42D06
:10114000B52DEAE5FDE50E94462D0E94772A85E14E
:101150000E948F285A924A928AE0A42DB52D8C9332
:1011600081E00E948F285A924A9289E1A42DB52DE0
:101170008C9381E00E948F285A924A9281E0A42D9C
:10118000B52D8C9381E00E948F285A924A9281E07B
:10119000A42DB52D8C9381E00E948F285A924A92FB
:1011A00081E0A42DB52D8C9381E00E948F285A9266
:1011B0004A928FEF9FEFA42DB52D8D939C9382E0E3
:1011C0000E948F285A924A928FEF9FEFA42DB52D3F
:1011D0008D939C9382E00E948F280E94C32060968A
:1011E0008EE10E948B28ECEEF1E00E941F2BE0E3E1
:1011F000FDE50E94462D0E94EE2B0E94F72B11F078
:101200000C945A095A924A92A42DB52DE0E7FDE5B7
:101210000E94462D0E94772A82E10E948F285A92CE
:101220004A928AE0A42DB52D8C9381E00E948F28EC
:101230005A924A9289E1A42DB52D8C9381E00E94A7
:101240008F285A924A9281E0A42DB52D8C9381E08B
:101250000E948F285A924A9281E0A42DB52D8C933A
:1012600081E00E948F285A924A9281E0A42DB52DE8
:101270008C9381E00E948F285A924A9280E098EFE6
:10128000A42DB52D8D939C9382E00E948F285A92B5
:101290004A928FEF9FEFA42DB52D8D939C9382E002
:1012A0000E948F280E94C32060968BE10E948B28A9
:1012B0000C945B0BECEEF1E00E941F2BE4E3FDE5E8
:1012C0000E94462D0E94EE2B0E94F72B11F00C94E9
:1012D000C1095A924A92A42DB52DE2E8FDE50E947B
:1012E000462D0E94772A83E10E948F285A924A92C3
:1012F0008AE0A42DB52D8C9381E00E948F285A920C
:101300004A9289E1A42DB52D8C9381E00E948F280B
:101310005A924A9281E0A42DB52D8C9381E00E94CF
:101320008F285A924A9281E0A42DB52D8C9381E0AA
:101330000E948F285A924A9281E0A42DB52D8C9359
:1013400081E00E948F285A924A9280E098EFA42D63
:10135000B52D8D939C9382E00E948F285A924A92D9
:101360008FEF9FEFA42DB52D8D939C9382E00E946B
:101370008F280E94C32060968CE10E948B280C94D9
:101380005B0BECEEF1E00E941F2BE8E3FDE50E9411
:10139000462D0E94EE2B0E94F72B11F00C94280A88
:1013A0005A924A92A42DB52DE6E9FDE50E94462DFC
:1013B0000E94772A82E10E948F285A924A928AE0FC
:1013C000A42DB52D8C9381E00E948F285A924A92C9
:1013D00089E1A42DB52D8C9381E00E948F285A922B
:1013E0004A9281E0A42DB52D8C9381E00E948F2834
:1013F0005A924A9281E0A42DB52D8C9381E00E94EF
:101400008F285A924A9281E0A42DB52D8C9381E0C9
:101410000E948F285A924A9280E098EFA42DB52D11
:101420008D939C9382E00E948F285A924A928FEF6C
:101430009FEFA42DB52D8D939C9382E00E948F2861
:101440000E94C32060968BE10E948B280C945B0B5A
:10145000ECEEF1E00E941F2BECE3FDE50E94462D2F
:101460000E94EE2B0E94F72B11F00C948F0A5A92D7
:101470004A92A42DB52DE8EAFDE50E94462D0E9472
:10148000772A83E10E948F285A924A928AE0A42DFB
:10149000B52D8C9381E00E948F285A924A9289E15F
:1014A000A42DB52D8C9381E00E948F285A924A92E8
:1014B00081E0A42DB52D8C9381E00E948F285A9253
:1014C0004A9281E0A42DB52D8C9381E00E948F2853
:1014D0005A924A9281E0A42DB52D8C9381E00E940E
:1014E0008F285A924A9280E098EFA42DB52D8D93C3
:1014F0009C9382E00E948F285A924A928FEF9FEF2E
:10150000A42DB52D8D939C9382E00E948F280E947C
:10151000C32060968CE10E948B280C945B0BECEE50
:10152000F1E00E941F2BE0E4FDE50E94462D0E94A1
:10153000EE2B0E94F72B11F00C94F60A5A924A9265
:10154000A42DB52DECEBFDE50E94462D0E94772AD7
:1015500085E10E948F285A924A928AE0A42DB52DE7
:101560008C9381E00E948F285A924A9289E1A42D9F
:10157000B52D8C9381E00E948F285A924A9281E087
:10158000A42DB52D8C9381E00E948F285A924A9207
:1015900081E0A42DB52D8C9381E00E948F285A9272
:1015A0004A9281E0A42DB52D8C9381E00E948F2872
:1015B0005A924A9280E098EFA42DB52D8D939C937A
:1015C00082E00E948F285A924A928FEF9FEFA42DBB
:1015D000B52D8D939C9382E00E948F280E94C3209A
:1015E00060968EE10E948B280C945B0BA7E5B1E01E
:1015F000E2EDFDE50E94462D0E94762E11F00C943E
:10160000070B80E090E0AAE2B2E08D939C935A929F
:101610004A92E7E5F1E0A42DB52D0E94562E80E117
:101620000E948F285A924A928AE0A42DB52D8C935D
:1016300081E00E948F285A924A9289E1A42DB52D0B
:101640008C9381E00E948F285A924A9281E0A42DC7
:10165000B52D8C9381E00E948F285A924A9281E0A6
:10166000A42DB52D8C9381E00E948F285A924A9226
:1016700081E0A42DB52D8C9381E00E948F285A9291
:101680004A9280E090E0A42DB52D8D939C9382E04A
:101690000E948F285A924A928FEF9FEFA42DB52D6A
:1016A0008D939C9382E00E948F280E94C3206096B5
:1016B00089E10E948B280C94AD0D0C3050E0150789
:1016C00011F00C94AD0DA7E5B1E00E940D2CEDE0FA
:1016D000F0E0A0E2B2E00E945B2EE4E4FDE50E94AF
:1016E000462D0E94EE2BE0E2F2E00E941F2B0E94AA
:1016F000B42BEDE0F0E0A0E2B2E00E945B2EE0E26D
:10170000F2E00E941F2BE0E2FDE50E94462D0E94C0
:10171000EE2B0E94F72B81E008F480E08F93E0E24B
:10172000F2E00E941F2BE8E4FDE50E94462D0E9496
:10173000EE2B0E94F72B81E010F009F080E09F91E2
:101740008923882311F40C94AD0B80E098EFAEE16F
:10175000B2E08D939C930C940F0CE0E2F2E00E94B7
:101760001F2BE8E4FDE50E94462D0E94EE2B0E940F
:10177000F72B81E008F480E08F93E0E2F2E00E9432
:101780001F2BECE4FDE50E94462D0E94EE2B0E94EB
:10179000F72B81E010F009F080E09F9189238823E6
:1017A00011F40C94DB0B86EC9CEFAEE1B2E08D9370
:1017B0009C930C940F0CE0E2F2E00E941F2BECE4EF
:1017C000FDE50E94462D0E94EE2B0E94F72B81E042
:1017D00008F480E08F93E0E2F2E00E941F2BE0E546
:1017E000FDE50E94462D0E94EE2B0E94F72B81E022
:1017F00010F009F080E09F918923882311F40C9464
:10180000090C80EE97E0AEE1B2E08D939C930C94CE
:101810000F0C80E090E0AEE1B2E08D939C93A7E5E1
:10182000B1E0E0E2F2E00E941F2B0E948829E7E588
:10183000F1E004E0A7E5B1E00E94682EE7E5F1E001
:10184000A2EFB1E012E0222701E033270E94022D2F
:10185000A2EFB1E00E94E128EAEDFDE50E94462DED
:101860000E94772A5A924A92E2EFF1E0A42DB52D18
:101870000E94562E85E10E948F285A924A9288E152
:10188000A42DB52D8C9381E00E948F285A924A9204
:1018900084E3A42DB52D8C9381E00E948F285A9269
:1018A0004A9281E0A42DB52D8C9381E00E948F286F
:1018B0005A924A9281E0A42DB52D8C9381E00E942A
:1018C0008F285A924A9281E0A42DB52D8C9381E005
:1018D0000E948F285A924A92AEE1B2E08D919C917B
:1018E000A42DB52D8D939C9382E00E948F285A924F
:1018F0004A928FEF9FEFA42DB52D8D939C9382E09C
:101900000E948F280E94C32060968EE10E948B283F
:10191000A4E2B2E00D911C91A6E2B2E04D915C917F
:10192000040F151FA8E2B2E00D931C93A8E2B2E0E9
:101930000D911C9142E050E00E94A728A8E2B2E07D
:101940004D935C93A8E2B2E00D911C91013050E000
:10195000150780E00CF481E08F93A8E2B2E00D91CE
:101960001C910F3F5FEF150780E014F009F081E054
:101970009F918923882311F40C94C40C80E090E09B
:10198000A8E2B2E08D939C93ACE2B2E0E8E2F2E030
:101990000E94D32DECE2F2E0A0E8BFE00E94562EB8
:1019A000E0E8FFE0ACE2B2E014E021E002E031E088
:1019B0000E94022DECE2F2E006E0ACE2B2E00E940E
:1019C000682EAAE2B2E04D915C91A8E2B2E00D91DE
:1019D0001C91041715071CF011F00C94F10C0C94D9
:1019E0004D0DA8E2B2E08D919C91AAE2B2E08D93F8
:1019F0009C935A924A92ECE2F2E0A42DB52D0E94FB
:101A0000562E85E10E948F285A924A9287E8A42D8B
:101A1000B52D8C9381E00E948F285A924A928AE3D6
:101A2000A42DB52D8C9381E00E948F285A924A9262
:101A300081E0A42DB52D8C9381E00E948F285A92CD
:101A40004A9281E0A42DB52D8C9381E00E948F28CD
:101A50005A924A9281E0A42DB52D8C9381E00E9488
:101A60008F285A924A9280E090E0A42DB52D8D9354
:101A70009C9382E00E948F285A924A928FEF9FEFA8
:101A8000A42DB52D8D939C9382E00E948F280E94F7
:101A9000C32060968EE10E948B28ACE2B2E00E94E7
:101AA000E128ECEDFDE50E94462D0E94772A5A922E
:101AB0004A92ECE2F2E0A42DB52D0E94562E85E16B
:101AC0000E948F285A924A9282E3A42DB52D8C93BE
:101AD00081E00E948F285A924A9286E2A42DB52D69
:101AE0008C9381E00E948F285A924A9281E0A42D23
:101AF000B52D8C9381E00E948F285A924A9281E002
:101B0000A42DB52D8C9381E00E948F285A924A9281
:101B100081E0A42DB52D8C9381E00E948F285A92EC
:101B20004A9280E090E0A42DB52D8D939C9382E0A5
:101B30000E948F285A924A928FEF9FEFA42DB52DC5
:101B40008D939C9382E00E948F280E94C320609610
:101B50008EE10E948B280C94AD0D789481E0481A98
:101B60008827580A22960895F894FFCFA8FFFF030C
:101B70002CFFFF095B084747010847470208474712
:101B800004084747020847470B4A4A782C79F479FA
:101B9000F4794BC39D98826399797900F479F41FA5
:101BA0004347470408474708084747020847470094
:101BB000084747000847084747014A4A782CF47904
:101BC000F44B986F4A4A04F89C79F4F4005E473469
:101BD000A2474706A2A20086084747124A4A0CFEBF
:101BE000C6219B21C6FE4A6FE39B9B00E36F694AB7
:101BF000FEE32121006F4A4A006F9B64D89B4A4A4A
:101C00001DC6216493D86F4AC6BED8D800234A4A5D
:101C1000232C79F499234A4A071B3F79F45EA04AA2
:101C20006B47470108474701003D4A3947470108CC
:101C30001E4809DC474704084747044A4A0CB9BD17
:101C40008EC18E28D8BAC088C1C100F37D646F19D7
:101C5000F5C16CBF6F64C08E8417194A4A1BFEF62B
:101C60007D8E84BB84212100C0C1171700286F4AD4
:101C70004A222CF44B234A4A096F53F41F4D4A253C
:101C800047470500FD4A39474701084E4A6935472D
:101C90004701084747074A4A0C7BBB1717027DF6E6
:101CA000C1171702BB196F0DBB171700C0E3281728
:101CB0001702B94A4A1B218E1717026CC610BB17B0
:101CC0001700BBBF694A4A222C79984A4A0392827C
:101CD000BCFE4A4A02F8791F374A3D4735094AFE99
:101CE000FA86003D4AC7E22F14AF6E4A4A006EA240
:101CF000B12F4AFE2D35752F1424692A4A4A0CC685
:101D0000C0171702BFFEBEC1171701BBBA4A6F7DCD
:101D1000177DE34A10C1171701B94A4A1CD8BB17EF
:101D20001701286F6F00107BD823FE4A4A232C4BE3
:101D30006F4A4A0282797900F47B4A4A03915E4DE8
:101D40004A6B43544A225D4A2F003D4A52FE4A04E0
:101D50008B584AFEAC116B4ADF3D4AACD14A4A006F
:101D6000694A2A4A4A0D9384171701F5C6FE8E1751
:101D700017020DFEE328BBF64A4A00238E1717010F
:101D8000B94A9B9310214A4A03FE5A10D8BAE34A33
:101D90004A03FE9BBAD8BAE34A4A01E36C1717011B
:101DA0007D6F4A4A00FE9B6410FE4A4A01C6239397
:101DB0009300BE6F4A4A192CE84A4A026F4B4B0205
:101DC000F45A4A4A025F1F374A3D114AFE04684AE4
:101DD0004A00D13D4A4A012D4783114A6975EB4AB1
:101DE0003D43974A69324A4A002D75354A4A0DE308
:101DF000F317170184BAE3C1171702C1E364C18E58
:101E0000214A4A00238E1717010D6488BB84289B42
:101E10004A4A016F196C8417C128644A4A01FEB905
:101E20006C841784F5BE4A4A00C6F51717017D6F0A
:101E3000FEBAC06CC1C100C64A4A005AC08EBBBBC4
:101E400000C17BE34A4A182C5F4A4A03FEFE034A5C
:101E50004A03925E4D4AFD4D4A4A00153D153D9795
:101E60003D4A4A016B35084E4A6983414A6E47B381
:101E70004A4A00974A4A00A24747004A4A0EB91701
:101E800017027DBF171704C07D177B4A4A01238EB6
:101E90001717018E6C171702BF4A4A00FEC01717AA
:101EA000008E19C1178EBE4A6FBF171700C1198E59
:101EB000178EBE4AC6881717017D6FBA841717019F
:101EC000BBC64A21F317170028BFBB17BDE34A4A18
:101ED000172C274A4A0D5A5E374A3DB34AFE08433B
:101EE000E2CDE53D4A223D4A2D084E4A4A00044DC6
:101EF0004A691EAF4A6BB34A4A001E4747004A4A26
:101F00000E9B84171704C1171704BB104A4A0123FC
:101F10008E17170128936C1717017D4A4A0064BB7E
:101F20001717008E938E171700C04A10C11717009D
:101F30008ED86C171700BF6FC6F51717017DFEE32B
:101F4000BD17170184E3FEBF1717017DB98417BBC6
:101F5000104A4A172CBC4A4A0D5A5E4D4A25B452C3
:101F60004AFE6B4AAC00FD4A3BA04A4A0034D14AC3
:101F70004A0197584A4A0239D14A4A001E47470047
:101F80004A4A0F28171703C193F31717038EE34A22
:101F90004A01238E171701B91B7D171701BD4A4A45
:101FA000007B17170284171701281BBF171702841D
:101FB0001717017D6FC6881717017D6F4A0D171718
:101FC00001BBC6E3F3171701BBBB00171700BB1912
:101FD0004A4A172C5F4A4A021BBC27BC27BCBC01DB
:101FE00027BC27825E8BCAC708B4B17F220447B4DE
:101FF0000424A2B4042473A9B1A72A35B4EB7A2A25
:102000003447A9CAC7864747004A4A0FBABB1717C1
:10201000027BFED8BB171702B9FE4A4A01238E176E
:102020001701B969C0171701844A4A002817170118
:10203000C1BF0D0D00B9236F7D171701C1BF0D0D75
:1020400000B9234AC6881717017DFE4A0D171701EC
:1020500084E39B8E171701880D0D01D8C64A4A17D5
:102060002CE84A4A021B4B79F47979065E830847CB
:1020700047010808024747000808004747000808CA
:1020800001470808014747000808014747000808BA
:10209000014747014A4A0FE3F5171702644A218EA8
:1020A000171701C1644A4A02BEC1171701B9FEC021
:1020B000171701844A4A000D171701F3C64A4A0050
:1020C0006F69FEB91717016CC64A4A006F694AC6A4
:1020D000F31717017D6F4A0D17170184E3C6F51733
:1020E0001701BFFE4A4A006F4A4A182C4B6F4A4AF2
:1020F0000227F47979009C239B9B0194C35E83475C
:1021000047204A4A10B9BB1717006CC64A4A000D4F
:10211000171701BDE34A4A021084171701C06F7DEB
:10212000171701BBE34A23BB171700BB0D23107B16
:10213000234A648E171700BB0D2364C0234A9B8E6D
:10214000171701F5C66FC0171701BBBE691917171E
:10215000018EF623D8BFC64A4A172CF45F4A4A03B9
:10216000E3BCBEFE4A4A02E34B1F834747204A4A6C
:10217000109B6C17BBB94A4A019B841784274A4AB3
:10218000026FBD171702BB27F3171702BFFE4A19CC
:1021900084171702BBBD214A691984171702BB288F
:1021A000E34ABF171703D8BA841717027D6FC6BD5D
:1021B000BB171702840D6F4A4A174F79F49B4A4A9E
:1021C000091B91791F7F1448C8484800C81448C8A3
:1021D000484800C81448C8484800C81448C8484877
:1021E00000C81448C8484800C81448C8484A4A109B
:1021F00069936C7D214A4A01FEB96CBFC64A4A0206
:10220000FE19288EC1F37B64B988846CBDF6FE4A42
:102210006F107D6C8EBD19E34A4A02937D6C8EBDB2
:10222000B9E34A4A0027288EC18E28BA23C0F3C1D9
:102230008EBDD81B4AE319BDC1F37D106F4A4A1801
:10224000E8F4F4004BF84A4A07E3C379F41F094A5B
:102250004A33FE21C64A4A036F216F4A4A04FEC62A
:10226000212100E36F4A6FE3212100C64A4A036F30
:10227000212100C6694A4A046F212100C6FE4A4A4C
:102280000169C6219B21C64A4A006F219B21C6696C
:102290004A4A01FEC62121006F4A4A1AE8797900AC
:1022A000F4796323FE4A4A02E45F4B797900F41F14
:1022B000584A4A9AE8F4F4037999C3E83F53F4F48E
:1022C000041F094A4A9A448C8C10144A4AFF4A4A0D
:1022D000FF4A4AFF4A4AFF4A4AFF4A4AFF4A4AFF20
:1022E0004A4AFF4A4AFF4A4AFF4A4AFF4A4AFF4AC5
:1022F0004AFF4A4AFF4A4AFF4A4AFF4A4AFF4A4AB5
:10230000FF4A4AFF4A4ACD0C0C2F4A4A0A0C0C28B5
:102310004A4A0A0C0C2F4A4A080C0C004A4A2F0C55
:102320000C004A4A060C0C004A4A280C0C004A4A87
:10233000060C0C004A4A2F0C0C004A4A050C4A4A6B
:10234000330C4A4A040C4A4A2C0C4A4A040C4A4AA6
:10235000330C4A4A030C4A4A350C4A4A020C4A4A90
:102360002E0C4A4A020C4A4A350C4A4A010C4A4A87
:1023700004FE33660BAE0B0B0076FE4A4A280C4A6D
:102380004A000C4A4A300C4A4A000C4A4A370C4A66
:102390004A000C4A4A0325AE0B2F6BFE25E0B038ED
:1023A0006B4A4A270C4A4A000C4A4A300C4A4A00F7
:1023B0000C4A4A07FEA0154A4A2B0C4A0C4A4A040A
:1023C0000BAE6B317777005D41C9360B4A4A28A0C6
:1023D0000C4A4A320C0C004A4A00FEFE004A4A04EB
:1023E000FE0C154A4A2C0CA04A4A0466B66B6B00D8
:1023F00049E058DF7AB5A54A4A280C0C004A4A320F
:102400000CA04A4A0060074A4A04544D544A4A2CD8
:102410000C0C004A4A04B2335633662D7633AD4C69
:102420000C4A4A28A00C4A4A32A00C4A4A00150C11
:10243000154A4A021B412E524A4A2CA00C4A4A0411
:1024400051CFFD6D0BD656E045F7714A4A280CA0D6
:102450004A4A320C0C004A4A017741694A4A016BE8
:10246000C90707004A4A2C0C0C004A4A04510505CA
:1024700000B7A10AA10A8581714A4A280C0C004ABA
:102480004A32A00C4A4A020C584A4A0215603D4A98
:102490004A2C0CA04A4A049405F03AA10AA10A85E4
:1024A00081CE4A4A280CA04A4A320CA04A4A02DF8E
:1024B000C96F4A4A320C0C004A4A04D670123A0AD2
:1024C0000A0016A1AA89614A4A28A00C4A4A320C7D
:1024D0000C004A4A02FE41604A4A32A00C4A4A04B1
:1024E000B6D66DC595AA9589B88A784A4A280C0C43
:1024F000004A4A320CA04A4A033D373D4A4A310C51
:102500000C004A4A0450B638805730573057597833
:102510004A4A28A00C4A4A32A00C4A4A04522E4A7F
:102520004A310CA04A4A04B65018D930D557305712
:1025300059904A4A280CA04A4A320C0C004A4A04D4
:102540006B0CDF4A4A300C0C004A4A0450187ED902
:10255000D5D5005730300040904A4A280C0C004A2C
:102560004A32A00C4A4A05D3AF4A4A30A00C4A4A24
:102570000450189AA630D557D5308F904A4A280C67
:10258000A04A4A320CA04A4A06C91C4A4A2F0C0CDF
:10259000004A4A04ABD762A6D5D4573040E6904AE9
:1025A0004A28A00C4A4A320C0C004A4A06DF0C6F3B
:1025B0004A4A2E0CA04A4A04509AEDA6D5D4573068
:1025C0004003904A4A280C0C004A4A320CA04A4A5E
:1025D00007DD524A4A2E0C0C004A4A04AB62A4574B
:1025E000D4D40057D58F03904A4A28A00C4A4A32C7
:1025F000A00C4A4A07314E604A4A2DA00C4A4A04B0
:10260000AB620E57D44057308F03D04A4A280CA0F3
:102610004A4A320C0C004A4A07076041DF4A4A2CFA
:102620000C4A0C4A4A032F7ED9574040005730408D
:1026300026484A4A270C4A0C4A4A32A04A0C4A4ABF
:10264000066037C43D4A4A2B0C4A4A000C4A4A04E9
:10265000FDA5CBF13042909F6E4A4A280C4A0C4AA5
:102660004A320C4A0C4A4A07411C4A4A2C0C4A4A34
:10267000010C4A4A350C4A4A000C4A4A320C4A4A72
:10268000000C4A4A06DD774A4A2B0C4A4A030C4A98
:102690004A330C4A4A010C4A4A320C4A4A010C4A53
:1026A0004A330C4A4A050C0C004A4A2F0C0C004ACB
:1026B0004A020C4A4A320C4A4A020C0C004A4A2F7F
:1026C0000C0C004A4A080CA0CE0CCE0CCE0CCE0C42
:1026D000A0CEA00CA00CA00CA00CA0A01A0C4A4AE2
:1026E000040C4A4A320C4A4A040CA0A02D0C4A4A57
:1026F0000A0CA0A0070C0C02A0A0010CA00C0C1C42
:102700004A4A040C4A4A320C4A4A040C0C2F4A4AE0
:1027100008A0A0004A4A0074E9E9001B4A4A03B233
:1027200087494A4A210C0C004A4A020C4A4A320C98
:102730004A4A020C0C004A4A2F0C0C004A4A05A0D7
:102740004A4A026A20A3544A4A02FE4696DF4A4A8F
:10275000230C4A4A010C4A4A320C4A4A010C4A4AA2
:10276000330C4A4A03A04A4A00694A696F9E1A1C00
:102770004A4A023DDAA3154A4A240C4A4A000C4A46
:102780004A320C4A4A000C4A4A350C4A4A01A04ACD
:102790004A05315C4649705470139E3CFE4A4A25F6
:1027A0000C4A0C4A4A32A04A0C4A4A370C4A4A00A0
:1027B0000C4A4A05742E674631F93C55550049FECE
:1027C0004A4A250C4A0C4A4A320C4A0C4A4A370CEF
:1027D0004AA04A4A05FE74466777FE4AFE1C41FC41
:1027E00070FE4A4A001B4A4A22A00C4A4A320C0C8C
:1027F000004A4A390C0C004A4A04FE493149F25851
:102800004A4A003D314954FC54CFB2FB4A4A220C9B
:102810000C004A4A320CA04A4A390CA04A4A03FE2C
:102820006AF954FE541C741B49311B4A3113CCFB0A
:102830007C4A4A22A00C4A4A32A00C4A4A39A00CCF
:102840004AE902701B6F02494A4A003D7C1C3D3C2C
:10285000494AFE492067F96F4A4A220CA04A4A3287
:102860000C0C004A4A390CA04A3E2B87E9F9465421
:102870004A4A01F2F2007046311B6A310731FE4AC2
:102880004A230C0C004A4A32A00C4A4A390C0C006C
:102890004A49FC9EC271551C741BFE1C20DADA00EA
:1028A0007CF9491B3158694A4A230CA04A4A320C28
:1028B000A04A4A390CA04A4A00FE6AFC2058741CFF
:1028C0003C3C00DA2020006713703DFE313100FEF1
:1028D0004A4A23A00C4A4A320C0C004A4A39A00C3E
:1028E0004A4A0254FC1BFE6A493C5CD2A071204952
:1028F000FEFE0031494A4A240C0C004A4A320CA020
:102900004A4A390CA04A4A00694A54463D4A4A009C
:102910001B49EA656500712EF94954467C74FE4AEC
:102920004A22A00C4A4A32A00C4A4A390C0C004AEE
:102930004A02DF7C3D4A1B497C208DD220543D3128
:1029400046CE5C7C704A4A220CA04A4A320C0C00EB
:102950004A4A390C0C004A4A00694A49136F74E923
:10296000F97413F2312E49FE153C313100FC494A0D
:102970004A220C0C004A4A32A00C4A4A39A0A00054
:102980004A4A02DFCCD34949003DFE3CF93D46317D
:102990004A3D3174693D6F4A4A220CA04A4A320CC2
:1029A000A04A4A390C0C004A4A0105465C55DF4AE8
:1029B0004A003D3C313D495870496AFE4A4A25A0CB
:1029C0000C4A4A320C0C004A4A390C0C004A15F9E0
:1029D0000F87DACC49FEFE006A313D4A15FCCC492E
:1029E000694A4A00694A4A230C0C004A4A320CA040
:1029F0004A4A390CA04AE9E701311B31FC497460AD
:102A0000494A6970CE20FE4A4A27A00C4A4A32A0A1
:102A10000C4A4A39A00C4A493C313D3D0054773CB0
:102A20002E0CCCF9F9001C67670070FE4A4A260C90
:102A3000A04A4A320C0C004A4A390C4A0CFDFD00EF
:102A4000151500545400DF5D675CF21C1C0049FC46
:102A50005C9E3D4AFE694A4A220C4A0C4A4A32A010
:102A60004A0C4A4A370C4A4A000C6A54540014541F
:102A700014153C019E7754151500DFF2463D4A4A75
:102A8000250C4A0C4A4A320C4A0C4A4A370C4A4A2C
:102A900001A0545400DF5454006E2E3EF215150070
:102AA0003D3D01153DFEFE004AFE4A4A210C4A4AC0
:102AB000000C4A4A320C4A4A000C4A4A350C4A4A2F
:102AC00002150C1554540131EA3E314A6FFE1BFECB
:102AD000FE044AFE4A4A1F0C4A4A010C4A4A320C7A
:102AE0004A4A010C4A4A330C4A4A050C0C004A4A2D
:102AF0002F0C0C004A4A020C4A4A320C4A4A020C79
:102B00000C004A4A2F0C0C004A4A080CA00CA0A04A
:102B10002B0C4A4A040C4A4A320C4A4A040CA0A024
:102B20002D0C4A4A0AA00CA00C0C2C4A4A040C4A50
:102B30004A320C4A4A040C0C2F4A4A080C0C004A30
:102B40004A2F0C0C004A4A020C4A4A320C4A4A02EA
:102B50000C0C004A4A2F0C0C004A4A050C4A4A0148
:102B600052414102584A4A2A0C4A4A010C4A4A3206
:102B70000C4A4A010C4A4A330C4A4A030C4A4A029C
:102B800006616102074A4A2B0C4A4A000C4A4A3243
:102B90000C4A4A000C4A4A350C4A4A010C4A4A037C
:102BA000B33B33256EE04A4A2C0C4A0C4A4A320C9D
:102BB0004A0C4A4A370C4A4A000C4A4A034EEB4C2C
:102BC000252FE04A4A2C0C4A0C4A4A320C4A0C4A3D
:102BD0004A370C4A0C4A4A044D6D766B2FE04A4A3C
:102BE0002DA00C4A4A32A00C4A4A390CA04A4A0489
:102BF000DEA776256EE04A4A2D0C0C004A4A320CBC
:102C00000C004A4A390C0C004A4A044E614C252FEC
:102C1000E04A4A2DA00C4A4A32A00C4A4A39A00C7C
:102C20004A4A043776AD25C8E04A4A2D0CA04A4AE4
:102C3000320CA04A4A390C0C004A4A044EEF762561
:102C400048E04A4A2D0C0C004A4A320C0C004A4A11
:102C5000390CA04A4A044D2D6D25C8E04A4A2D0C76
:102C6000A04A4A320CA04A4A390C0C004A4A044E87
:102C7000EFEE25FA074A4A2DA00C4A4A32A00C4A28
:102C80004A39A00C4A4A044E4CFA25FADD4A4A0752
:102C9000694A4A230C0C004A4A320C0C004A4A3951
:102CA0000C0C004A4A04DEEE2D2509DD4A4A07696C
:102CB0004A4A23A00C4A4A32A00C4A4A390CA04A7C
:102CC0004A04DE3BA7256DDD4A4A2D0CA04A4A3254
:102CD0000CA04A4A390C0C004A4A044E4C7625FA9C
:102CE000DD4A4A2D0C0C004A4A320C0C004A4A3983
:102CF000A00C4A4A04DEA72D25FA2E4A4A2D0CA024
:102D00004A4A320CA04A4A390C0C004A4A044E4C3A
:102D10007A2509DD4A4A2DA00C4A4A32A00C4A4ABB
:102D2000390CA04A4A04DEE1762509DD4A4A2D0C19
:102D30000C004A4A320C0C004A4A390C0C004A4A30
:102D400004DEEFA725FA3752520244525201F252E2
:102D50005201DF4A4A20A00C4A4A32A00C4A4A39A2
:102D6000A00C4A4A0468DD6D256E667A7A02662DEB
:102D70002D01662D2D00EF414A4A200CA04A4A320F
:102D80000CA04A4A390C4A0C4A4A03DE7AAD256B3C
:102D90002525016B6B00256B6B002525006B6B00F7
:102DA000CA414A4A1F0C4A4A000C4A4A300C4A4A55
:102DB000000C4A4A370C4A4A000C4A4A03DEEFA785
:102DC000254A4A03694A694A4A01696B3B414A4AB2
:102DD0001F0C4A4A000C4A4A300C4A4A000C4A4A24
:102DE000370C4A4A010C4A4A02682D6DFAFA050965
:102DF000FA6DFA6D6D0161414A4A1E0C4A4A020C95
:102E00004A4A2E0C4A4A020C4A4A350C4A4A030CDA
:102E10004A4A0129B3B30E06F24A4A1D0C4A4A0433
:102E20000C4A4A2C0C4A4A040C4A4A330C4A4A05BA
:102E30000C0C004A4A2F0C0C004A4A060C0C004AA3
:102E40004A280C0C004A4A060C0C004A4A2F0C0C6B
:102E5000004A4A080CA00CA00CA00CA00CA00CA0CE
:102E60000CA00CA00CA00CA00CA00CA00CA00CA002
:102E70000CA00CA00CA00CA00CA00CA00CA00CA0F2
:102E80000CA00CA00C4A4A0A0CA00CA00CA00CA090
:102E90000CA00CA00CA00CA00CA00CA00CA00CA0D2
:102EA0000CA00CA00CA00CA00CA00CA00CA00CA0C2
:102EB0000CA04A4A0A0CA00CA00CA00CA00CA00C60
:102EC000A00CA00CA00CA00CA00CA00CA00CA00CA2
:102ED000A00CA00CA00CA00CA00CA00CA00CA00C92
:102EE000A00CA00CA00C4A4A040011489C0BCE1563
:102EF000086E7455FF184208A5341A6FC63AA282AC
:102F00009D3B8410FBAE4276B4EFFD345B4FFEB6C2
:102F1000BD94CEBBE73CB303F800741CFC307B08C7
:102F2000F79DCE3729714352B1019CB0FEBAADB8BE
:102F3000FE388CD4E73E4A92FCF3FA285AEC8D38DE
:102F400093A9A9C6B5B9AD12D6BC2173D6784A8B60
:102F5000C63D53B332F16B9673AF94BB7CD7DC6A3A
:102F60008433C5F5EF5D838AF309191194B24233B6
:102F7000222DBD54D5B5B5732290C67BDEB9FFFFB7
:102F8000E9A29CB5738F632DCA888C9CF634AD760C
:102F9000F225DEDBA4D1B5DD31B4CE792151FE9925
:102FA00081A8942EB5B6B0E0F490BDF77BD15B3A22
:102FB000F38BFDB65268AD5B946F6B6FF7BFE6FAAB
:102FC000EF5FF965BDFADEDCFF7DE6D97B6C19AAFF
:102FD0007475EF3B32AEC63CC6386333E941AD7819
:102FE000FB0CC593FAAA73FA9D164AB7A306F42EF2
:102FF0001A2EF8A2C3A73312ACAEF9C7A3AC421184
:10300000426B8ACA7B8CF92410D15B12F287FDD502
:10301000FCB2EE76C42A836952EDF46FE9C3639B78
:10302000FE79F246F3EDACF18C767BF0B2E34B9394
:1030300093EB4A9894D83A159CF671EA11ABBBC849
:10304000847CADFACE7D9CFB847384365350E63687
:103050004A6A118A635894DCDCAB8B90FBEFFD75F8
:10306000F861FD32FA69FDF7FB6DFAEBF8E38BECE2
:10307000F2C87C11CCEFFF3C7CD6CE7C8C51949571
:1030800052F4AD3263F28BEEFF5A6B933A2A732AF5
:10309000C5F619121952A55C6BDBFC714A97A4D0D6
:1030A0003B112AB19CF46B4ED6BAB597A51763D3E2
:1030B000FEFBFF1B198910AF9BEAF34ACDF5944E36
:1030C0007BF121EA52F89CF78C54FEF731B1B574CC
:1030D000F986E961F9E7FCD3ABCBFE16CE36C63BE9
:1030E000B510BDB5E73DFFBE99C781E00E948229BA
:1030F00082E00E94822980914802AA81BB818C9340
:1031000080E08093480280E08093410280E08093D9
:10311000430283E8809342028FEA809344020E9434
:10312000D2188FEF809359028FEF80935A028FEF5E
:1031300080935B028FEF80935C028FEF80935D0240
:103140008FEF80935E028FEF80935F028FEF80930B
:10315000600281E090E0A881B9818D939C93A88161
:10316000B9810D911C91003B56E1150718F011F043
:103170000C94C61898E0A9E5B2E00E945529A881F0
:10318000B9810E94932810F40C94AF18C59AAA81B3
:10319000BB818C918093480283E0481A8827580AA3
:1031A000249608958CE090E0A9EBB3E08D939C9376
:1031B0008FEE8093590288E080935A0288E18093D1
:1031C0005B0282E180935D0285E180935F0283E18F
:1031D0008093610286E1809363020091480200308F
:1031E00011F00C94F81880E080935C020C946D1937
:1031F000023011F00C941D1983E080935C0203E807
:1032000040914102041BA1E4B2E00C9303E8409119
:103210004202041BA2E4B2E00C930FEA4091430285
:10322000041BA3E4B2E00C930FEA40914402041B98
:10323000A4E4B2E00C930C946D19013011F00C94DD
:10324000461985E080935C0203E840914302041B29
:10325000A3E4B2E00C9303E840914402041BA4E40D
:10326000B2E00C93009141028091430280934102AD
:10327000A3E4B2E00C930091420280914402809357
:103280004202A4E4B2E00C930C946D19033011F0E7
:103290000C946D1986E080935C020FEA4091410224
:1032A000041BA1E4B2E00C930FEA40914202041B1C
:1032B000A2E4B2E00C93009141028091430280931A
:1032C0004102A3E4B2E00C930091420280914402D7
:1032D00080934202A4E4B2E00C9380914102809377
:1032E0005E0280914202809360028091430280934B
:1032F00062028091440280936402C69A0E94ED2388
:10330000C598C698089582E00E94822982E00E94B2
:10331000822981E00E94822981E00E94822981E045
:103320008093500280E090E0AEE4B2E08D939C93F5
:10333000AE85BF858C9180934102AC85BD858C9113
:1033400080934302AA85BB858C9180934202A88515
:10335000B9858C91809344020E94D218AA85BB85BE
:103360000C91AE85BF854C91041BAA81BB810C9347
:10337000AA81BB818C918F5F8C93A885B9850C91B4
:10338000AC85BD854C91041BA881B9810C93A881A3
:10339000B9818C918F5F8C93AA81BB810D9111278C
:1033A000A881B9814D9155270E946D2AAC81BD81BC
:1033B0000D931C9381E090E0AE81BF818D939C932F
:1033C000AC81BD814D915C91AE81BF810D911C910D
:1033D0000417150718F011F00C94FC190E94031A39
:1033E00092E0A9E5B2E00E945529AE81BF810E941A
:1033F000932810F40C94E019C59A86E0481A88279F
:10340000580A2896089581E00E94822981E00E944E
:10341000822981E00E94822982E00E94822982E042
:103420000E94822900914D02003011F00C942C1A58
:103430000E948428A9E5B2E00E94E42B0C920E942D
:103440007E280E948428AAE5B2E00E94E42B0C9218
:103450000E947E280C94B61B013011F00C94E41AE3
:10346000AEE4B2E00D911C91003050E0150711F070
:103470000C94DE1A00915002013011F00C94571A8E
:103480000E948428A9E5B2E00E94E42B0C920E94DD
:103490007E280E948428AAE5B2E00E94E42B0C92C8
:1034A0000E947E2880E0809350020C94DC1AA9E5EB
:1034B000B2E08C91AA81BB818D9388278C9398E090
:1034C000AA81BB810E949F2AAA81BB810D911C9178
:1034D000AAE5B2E04D915527040F151FAA81BB81C3
:1034E0000D931C930E948428A9E5B2E00E94E42B6E
:1034F0000C920E947E280E948428AAE5B2E00E94D5
:10350000E42B0C920E947E28A9E5B2E08C91A88160
:10351000B9818D9388278C9398E0A881B9810E9406
:103520009F2AA881B9810D911C91AAE5B2E04D9125
:103530005527040F151FA881B9810D931C93AA81EB
:10354000BB814D915C91A881B9810D911C910417AB
:10355000150711F00C94DC1A0E948428AC81BD81FF
:103560000E94E42B0C920E947E28AC81BD818C913C
:10357000AEE4B2E08D9388278C9398E0AEE4B2E09D
:103580000E949F2A0E948428AC81BD810E94E42B66
:103590000C920E947E28AEE4B2E00D911C91AC81A9
:1035A000BD814D915527040F151FAEE4B2E00D9378
:1035B0001C9381E0809350020C94E21AAEE4B2E0D6
:1035C0000E949A280C94B61B023011F00C94F51A44
:1035D0000E948428A5E4B2E00E94E42B0C920E9491
:1035E0007E280E94E51B0C94B61B033011F00C944E
:1035F0004E1BAEE4B2E00D911C91003050E0150777
:1036000011F00C94481B00915002013011F00C9401
:10361000191B0E948428A5E4B2E00E94E42B0C92BE
:103620000E947E280E94E51B80E0809350020C944B
:10363000461B80914502AC81BD818C930E948428F9
:10364000A5E4B2E00E94E42B0C920E947E280E9426
:10365000E51B40914502AC81BD810C91041711F02E
:103660000C94461B0E948428AC81BD810E94E42BEF
:103670000C920E947E28AC81BD818C91AEE4B2E0B8
:103680008D9388278C9381E0809350020C944C1B7F
:10369000AEE4B2E00E949A280C94B61B043011F0FC
:1036A0000C945F1B0E948428A5E4B2E00E94E42BE6
:1036B0000C920E947E280E94BC1B0C94B61B053005
:1036C00011F00C94B61BAEE4B2E00D911C910030E9
:1036D00050E0150711F00C94B21B0091500201301C
:1036E00011F00C94831B0E948428A5E4B2E00E9490
:1036F000E42B0C920E947E280E94BC1B80E08093E9
:1037000050020C94B01B80914502AC81BD818C931A
:103710000E948428A5E4B2E00E94E42B0C920E944F
:103720007E280E94BC1B40914502AC81BD810C915A
:10373000041711F00C94B01B0E948428AC81BD8149
:103740000E94E42B0C920E947E28AC81BD818C915A
:10375000AEE4B2E08D9388278C9381E08093500291
:103760000C94B61BAEE4B2E00E949A2887E0481A97
:103770008827580A2A960895A5E4B2E00D911127EA
:1037800042E050E00E946D2AA6E4B2E00D931C9343
:10379000EAEEFEE20E94462DA6E4B2E08D919C91F5
:1037A000A9E5B2E00E94EF2CA6E4B2E00E949328C3
:1037B000EAEEFEE20E94462DA6E4B2E08D919C91D5
:1037C000AAE5B2E00E94EF2C089581E00E948229D0
:1037D00081E00E94822981E00E94822980E0AC8100
:1037E000BD818C9380E0AA81BB818C9380E0A8810D
:1037F000B9818C93A5E4B2E08C9181FBAC81BD8151
:103800008C9181F98C93A5E4B2E08C9180FBAC8122
:10381000BD818C9180F98C93A5E4B2E08C9184FBFE
:10382000AA81BB818C9182F98C93A5E4B2E08C9142
:1038300083FBAA81BB818C9181F98C93A5E4B2E0D2
:103840008C9182FBAA81BB818C9180F98C93A5E439
:10385000B2E08C9187FBA881B9818C9182F98C931D
:10386000A5E4B2E08C9186FBA881B9818C9181F9A5
:103870008C93A5E4B2E08C9185FBA881B9818C91F1
:1038800080F98C93AC81BD810C914AE0049F0C922D
:10389000AA81BB810C9149E0049F0C92A881B98157
:1038A0000C9144E0049F0C92AC81BD810C910E31CF
:1038B00011F00C945F1C8FE1AC81BD818C93A881C9
:1038C000B9810C910C3111F00C946A1C8FE1A88124
:1038D000B9818C93A881B9818C918093590293E02E
:1038E000A9E5B2E00E94972AAA81BB818C9187FB4F
:1038F000A9E5B2E08C9182F98C93AA81BB818C916D
:1039000086FBA9E5B2E08C9181F98C93AA81BB81F9
:103910008C9185FBA9E5B2E08C9180F98C93AA810A
:10392000BB818C9180935A0293E0AAE5B2E00E9499
:10393000972A00915A02AC81BD814C91040FAAE5EF
:10394000B2E00C9383E0481A8827580A2696089517
:1039500082E00E94822982E00E94822981E00E9406
:10396000822981E00E948229A889B9898C9180935B
:103970004102AE85BF858C9180934302AC85BD85A5
:103980008C9180934202AA85BB858C9180934402DE
:103990000E94D218AC85BD850C91A889B9894C913B
:1039A000041BAA81BB810C93AA81BB818C918F5F80
:1039B0008C93AA85BB850C91AE85BF854C91041B69
:1039C000A881B9810C93A881B9818C918F5F8C9368
:1039D000AA81BB810D911127A881B9814D915527ED
:1039E0000E946D2AAC81BD810D931C93A885B98579
:1039F0008D919C91A9E4B2E08D939C930E947423D5
:103A000081E090E0AE81BF818D939C93AC81BD81BC
:103A10004D915C91AE81BF810D911C9104171507EA
:103A200018F011F00C94201D92E0A9E5B2E00E947C
:103A30005529AE81BF810E94932810F40C94061D75
:103A4000C59A86E0481A8827580A289608955A92F7
:103A50004A92AC85BD858C91A42DB52D8C9381E0C7
:103A60000E948F285A924A92AC85BD858C91A42DD4
:103A7000B52D8C9381E00E948F285A924A92AC8592
:103A8000BD858C91A42DB52D8C9381E00E948F284B
:103A90005A924A92A889B9898C91A42DB52D8C93FC
:103AA00081E00E948F285A924A92AC85BD858C9104
:103AB000A42DB52D8C9381E00E948F285A924A92B2
:103AC000AC85BD858D919C91A42DB52D8D939C9336
:103AD00082E00E948F280E94BA1E2C9687E00E94E6
:103AE0008B285A924A92A885B9858C91A42DB52D20
:103AF0008C9381E00E948F285A924A92AC85BD85B2
:103B00008C91A42DB52D8C9381E00E948F285A9220
:103B10004A92AC85BD858C91A42DB52D8C9381E006
:103B20000E948F285A924A92AC85BD858C91A42D13
:103B3000B52D8C9381E00E948F285A924A92AC85D1
:103B4000BD858C91A42DB52D8C9381E00E948F288A
:103B50005A924A92AC85BD858D919C91A42DB52D2C
:103B60008D939C9382E00E948F280E94BA1E2C960F
:103B700087E00E948B285A924A92AC85BD858C9131
:103B8000A42DB52D8C9381E00E948F285A924A92E1
:103B9000A885B9858C91A42DB52D8C9381E00E94C8
:103BA0008F285A924A92AC85BD858C91A42DB52D53
:103BB0008C9381E00E948F285A924A92AC85BD85F1
:103BC0008C91A42DB52D8C9381E00E948F285A9260
:103BD0004A92AC85BD858C91A42DB52D8C9381E046
:103BE0000E948F285A924A92AC85BD858D919C91F6
:103BF000A42DB52D8D939C9382E00E948F280E9466
:103C0000BA1E2C9687E00E948B285A924A92AC8565
:103C1000BD858C91A42DB52D8C9381E00E948F28B9
:103C20005A924A92AC85BD858C91A42DB52D8C936A
:103C300081E00E948F285A924A92A889B9898C9172
:103C4000A42DB52D8C9381E00E948F285A924A9220
:103C5000AC85BD858C91A42DB52D8C9381E00E94FF
:103C60008F285A924A92AC85BD858C91A42DB52D92
:103C70008C9381E00E948F285A924A92AC85BD8530
:103C80008D919C91A42DB52D8D939C9382E00E94E3
:103C90008F280E94BA1E2C9687E00E948B280895D8
:103CA00081E00E94822981E00E948229AA85BB8549
:103CB0008C9180934102A885B9858C9180934302B1
:103CC000AE81BF810C91013011F00C947D1EAA854C
:103CD000BB850C9141E0040FA2E4B2E00C93A885EF
:103CE000B9850C9141E0040FA4E4B2E00C9384E0A8
:103CF000A881B9818C930C948B1EAA85BB858C916D
:103D000080934202A885B9858C918093440281E01A
:103D1000A881B9818C930E94D218AC81BD818D910C
:103D20009C91A9E4B2E08D939C930E94742381E05E
:103D3000AA81BB818C93A881B9814C91AA81BB8156
:103D40000C91041718F011F00C94B31E92E0A9E541
:103D5000B2E00E945529AA81BB818C918F5F8C9320
:103D600010F40C949B1EC59A82E0481A8827580AC2
:103D70002496089582E00E94822982E00E9482298E
:103D800082E00E94822982E00E94822982E00E94D1
:103D9000822982E00E94822982E00E94822981E0B9
:103DA0000E94822981E00E948229AC8DBD8D8C9178
:103DB000AA81BB818C93AA8DBB8D8C91A881B9817E
:103DC0008C9380E090E0A885B9858D939C93A88D15
:103DD000B98D0D911127AC8DBD8D4D915527041BCB
:103DE000150BA889B9890D931C93AE89BF890D91D4
:103DF0001127AA8DBB8D4D915527041B150BAE8540
:103E0000BF850D931C9381E090E0AC85BD858D93BB
:103E10009C9381E090E0AA85BB858D939C93A889B3
:103E2000B9890D911C91003050E015070CF402C0C7
:103E30000C942C1F8FEF9FEFAC85BD858D939C93C9
:103E4000A889B9890D911C914FEF5FEF0E946D2AEF
:103E5000A889B9890D931C93AE85BF850D911C91DE
:103E6000003050E015070CF402C00C94491F8FEF8E
:103E70009FEFAA85BB858D939C93AE85BF850D91E1
:103E80001C914FEF5FEF0E946D2AAE85BF850D93A9
:103E90001C93A889B9894D915C91AE85BF850D9120
:103EA0001C91041715071CF011F00C94F11F02E08F
:103EB00010E0A889B9894D915C910E946D2AAE816C
:103EC000BF810D931C9302E010E0AE85BF854D913C
:103ED0005C910E946D2AAC81BD810D931C93A88DCD
:103EE000B98D4C91AA81BB810C91041711F40C94EB
:103EF000EF1F5A924A92AC81BD818C91A42DB52DB1
:103F00008C9381E00E948F285A924A92AC81BD81A5
:103F10008C91A42DB52D8C9381E00E948F285A920C
:103F20004A92AA8DBB8D8C91A42DB52D8C9381E0E6
:103F30000E948F285A924A92AA8DBB8D8D919C9196
:103F4000A42DB52D8D939C9382E00E948F280E9412
:103F5000501E289685E00E948B28AA81BB810C9177
:103F6000AC85BD854C91040FAA81BB810C93A885BB
:103F7000B9850D911C91AC81BD814D915C91040F6F
:103F8000151FA885B9850D931C93A889B9894D91F2
:103F90005C91A885B9850D911C91041715071CF03B
:103FA00011F00C94D51F0C94ED1FA881B9810C91D0
:103FB000AA85BB854C91040FA881B9810C93A88573
:103FC000B9850D911C91AE81BF814D915C91041B0F
:103FD000150BA885B9850D931C930C946F1F0C9439
:103FE000892002E010E0AE85BF854D915C910E9472
:103FF0006D2AAE81BF810D931C9302E010E0A88969
:10400000B9894D915C910E946D2AAC81BD810D935F
:104010001C93AE89BF894C91A881B9810C9104177A
:1040200011F40C9489205A924A92AC81BD818C91F2
:10403000A42DB52D8C9381E00E948F285A924A922C
:10404000AC81BD818C91A42DB52D8C9381E00E9413
:104050008F285A924A92AA8DBB8D8C91A42DB52D92
:104060008C9381E00E948F285A924A92AA8DBB8D30
:104070008D919C91A42DB52D8D939C9382E00E94EF
:104080008F280E94501E289685E00E948B28A881C8
:10409000B9810C91AA85BB854C91040FA881B98187
:1040A0000C93A885B9850D911C91AC81BD814D9172
:1040B0005C91040F151FA885B9850D931C93AE85DF
:1040C000BF854D915C91A885B9850D911C91041710
:1040D00015071CF011F00C946F200C948720AA8116
:1040E000BB810C91AC85BD854C91040FAA81BB812D
:1040F0000C93A885B9850D911C91AE81BF814D911E
:104100005C91041B150BA885B9850D931C930C9429
:1041100009205A924A92AC81BD818C91A42DB52D73
:104120008C9381E00E948F285A924A92AC81BD8183
:104130008C91A42DB52D8C9381E00E948F285A92EA
:104140004A92AA8DBB8D8C91A42DB52D8C9381E0C4
:104150000E948F285A924A92AA8DBB8D8D919C9174
:10416000A42DB52D8D939C9382E00E948F280E94F0
:10417000501E289685E00E948B2880E1481A8827E7
:10418000580A6296089581E00E94822981E00E9487
:10419000822981E00E94822981E00E94822981E0B7
:1041A0000E94822982E00E94822981E00E94822965
:1041B00081E00E94822981E00E94822982E00E949F
:1041C000822981E00E94822982E00E94822982E085
:1041D0000E94822981E00E94822981E00E94822936
:1041E00081E00E94822981E00E948229AAA5BBA5C4
:1041F0000C9144E0049FA8A1B9A10C92A8A1B9A177
:104200008C9183508C93A8A1B9A1AD90BB24A0E55B
:10421000B2E0AA0DBB1D8C91AE8DBF8D8C93A8A171
:10422000B9A18C918F5F8C93A8A1B9A1AD90BB244B
:10423000A0E5B2E0AA0DBB1D8C91AE85BF858D9324
:1042400088278C93AE85BF850C91AEA1BFA14C9100
:10425000049FAC8DBD8D0C92A8A1B9A18C918F5FEC
:104260008C93A8A1B9A1AD90BB24A0E5B2E0AA0DA2
:10427000BB1D8C91AA8DBB8D8C93AA8DBB8D0C918F
:10428000A8A5B9A54C91049FAA8DBB8D0C92A8A19D
:10429000B9A18C918F5F8C93A8A1B9A1AD90BB24DB
:1042A000A0E5B2E0AA0DBB1D8C91A88DB98D8C93B1
:1042B000A88DB98D0C91AEA1BFA14C91049FA88D82
:1042C000B98D0C9281E0AC85BD858C93A8A9B9A964
:1042D0000E94702E482FAC85BD850C91041718F0F4
:1042E00011F00C946E23AC85BD858C91E8A9F9A9D9
:1042F00001E00A93AB85BC850E94612EAA85BB852F
:104300008C91AE89BF898D9388278C93AE89BF89A4
:104310000D911C910A3750E0150718F011F00C941C
:1043200093210C94F721AE89BF890D911C91043E15
:1043300050E0150711F00C94A5218FE790E0AE89AD
:10434000BF898D939C930C94F721063F50E015078D
:1043500011F00C94B32180E890E0AE89BF898D9371
:104360009C930C94F7210C3F50E0150711F00C942E
:10437000C12181E890E0AE89BF898D939C930C9414
:10438000F721043C50E0150711F00C94CF2182E88E
:1043900090E0AE89BF898D939C930C94F721063DE4
:1043A00050E0150711F00C94DD2183E890E0AE8910
:1043B000BF898D939C930C94F7210C3D50E0150719
:1043C00011F00C94EB2184E890E0AE89BF898D93C5
:1043D0009C930C94F7210F3D50E0150711F00C94BD
:1043E000F72185E890E0AE89BF898D939C93AE89D3
:1043F000BF890D911C9140E250E0041B150BAE8962
:10440000BF890D931C93AE85BF850D911C91AE891C
:10441000BF894D915C910E946D2AAE89BF890D9331
:104420001C93AC85BD850C9141E0041BAC89BD8912
:104430000C93AC89BD890C91AA8DBB8D4C91049FC6
:10444000A1E4B2E00C9200914102AEA5BFA54C914F
:10445000040FA1E4B2E00C93ACA5BDA58C918093B0
:104460004302AA8DBB8D0C9140914102040FA2E43E
:10447000B2E00C93809142028150809342020091FD
:104480004302A88DB98D4C91040FA4E4B2E00C93C3
:10449000809144028150809344020E94D21880E0AF
:1044A00090E0A885B9858D939C93AE85BF854D918D
:1044B0005C91A885B9850D911C910417150718F01A
:1044C00011F00C946523AAA5BBA50C91013011F045
:1044D0000C947822E8E3F8E40E94462DAE89BF8967
:1044E0008D919C91ABE4B2E00E94EF2C0C94882259
:1044F000023011F00C948822E8E6FBE40E94462D7D
:10450000AE89BF898D919C91ABE4B2E00E94EF2C03
:1045100081E0AE81BF818C93AEA1BFA14C91AE81F1
:10452000BF810C91041718F011F00C945A23AE853A
:10453000BF854D915C91A885B9850D911C9104179B
:10454000150711F00C94A72280E080934B02A8A1DC
:10455000B9A1AD90BB24AFE4B2E0AA0DBB1D0C9194
:10456000A8A1B9A1AD90BB24ADE4B2E0AA0DBB1DDA
:104570004C91041BAC81BD810C93AC81BD810C912D
:10458000A8A5B9A54C91049FAC81BD810C9281E096
:1045900080934C02AC81BD814C9100914C02041778
:1045A00018F011F00C94EB22AAA1BBA18D919C9163
:1045B000A9E4B2E08D939C930E94742392E0A9E554
:1045C000B2E00E945529ACE4B2E08C918F5F8C93ED
:1045D00010F40C94CA22AE8DBF8D0C9141E0041BE7
:1045E000AC81BD810C93AC81BD818C9180934C02D8
:1045F00040914C0200E0041718F011F00C94522383
:1046000081E0AA81BB818C93A8A5B9A54C91AA8110
:10461000BB810C91041718F011F00C944A23ACE400
:10462000B2E08C91ABE4B2E00E94FC2C0E94F22C30
:104630000C900822689409F4E894A881B98188272D
:1046400080F98C93A881B9810C91013011F00C9400
:104650003323ACA1BDA18D919C91A9E4B2E08D93CF
:104660009C930C943B23AAA1BBA18D919C91A9E49E
:10467000B2E08D939C930E94742392E0A9E5B2E08E
:104680000E945529AA81BB818C918F5F8C9310F475
:104690000C94042380914C02815080934C0210F0C2
:1046A0000C94F822AE81BF818C918F5F8C9310F4B3
:1046B0000C948C22AE89BF890E949328A885B98565
:1046C0000E94932810F40C945522C59AAC85BD85A0
:1046D0008C918F5F8C9310F40C94662185E1481ABD
:1046E0008827580AA29608958091490280935A0219
:1046F00098E0A9E4B2E00E94AA2A8091490280933E
:10470000590208958CE291E00E947329C4988BE4C9
:1047100090E00E947329C5988BE490E00E94732971
:10472000C1988BE490E00E947329C69A8BE490E0D4
:104730000E947329C49A8BE490E00E947329EEEEE4
:10474000F7E40E94462D0E947E2881E0809341027A
:1047500000914102053218F011F00C94D1230E940F
:104760008428A6E4B2E00E94DF2C0E947E28A6E402
:10477000B2E00D911C91003050E3150711F00C943C
:10478000C7238BE490E00E9473290C94C9230E94F4
:10479000D423A1E4B2E08C918F5F8C9310F40C943D
:1047A000A823C59AC6980895C69AC59898E0A6E425
:1047B000B2E00E948A2A91E0A6E4B2E00E94552964
:1047C00098E0A6E4B2E00E947D2A91E0A6E4B2E07F
:1047D0000E945529C59AC6980895C598A9EBB3E0DB
:1047E0009C91A9E5B2E00E945529C59A0895FDFD66
:1047F000FDFD003000EF04EE041BFEFEFEFE90EF18
:10480000044A3F7F04EE0643003090EF830900081E
:10481000AF0B000A00050006000700EF0CEE90EF5A
:104820008000B0EF024900EF017F81E102E276E211
:1048300083E1018090EF0000000000000000000014
:10484000040E0E04040004001B1B120000000000F4
:10485000000A1F0A0A1F0A00080E100C021C04009E
:1048600019190204081313000814140815120D0076
:104870000C0C0800000000000408080808080400E8
:104880000804040404040800000A0E1F0E0A0000B5
:104890000004041F0404000000000000000C0C08C9
:1048A0000000001F0000000000000000000C0C00D1
:1048B00000010204081000000E11131519110E005A
:1048C000040C040404040E000E11010608101F005D
:1048D0000E11010E01110E0002060A121F02020043
:1048E0001F10101E01110E000608101E11110E00DF
:1048F0001F010204080808000E11110E11110E000C
:104900000E11110F01020C0000000C0C000C0C0029
:1049100000000C0C000C0C08020408100804020033
:1049200000001F00001F000008040201020408002C
:104930000E110106040004000E11171517100E00C9
:104940000E11111F111111001E11111E11111E0047
:104950000E11101010110E001E11111111111E0058
:104960001F10101E10101F001F10101E101010001E
:104970000E11101711110F001111111F111111003B
:104980000E04040404040E000101010111110E00C3
:1049900011121418141211001010101010101F0012
:1049A000111B1511111111001119151311111100FD
:1049B0000E11111111110E001E11111E10101000F8
:1049C0000E11111115120D001E11111E12111100E0
:1049D0000E11100E01110E001F0404040404040043
:1049E0001111111111110E0011111111110A0400F0
:1049F0001111151515150A0011110A040A111100DB
:104A00001111110A040404001E02040810101E00F3
:104A10000E08080808080E00001008040201000033
:104A20000E02020202020E00040A11000000000041
:104A3000000000000000001F0C0C0400000000003B
:104A400000000E010F110F0010101E1111111E0099
:104A500000000E1110110E0001010F1111110F00B5
:104A600000000E111F100E000608081E080808009E
:104A700000000F11110F010E10101C121212120063
:104A80000400040404040400020006020202120CE2
:104A90001010121418141200040404040404060074
:104AA00000001A151511110000001C12121212003C
:104AB00000000E1111110E0000001E1111111E1028
:104AC00000000F1111110F010000160908081C0049
:104AD00000000E100E010E0000081E08080A040057
:104AE0000000121212160A0000001111110A04002F
:104AF00000001111151F0A00000012120C12120002
:104B000000001212120E041800001E020C101E00EB
:104B10000608081808080600040404040404040035
:104B20000C02020302020C00000000000000000062
:104B30000A000E010F110F000A000E1111110E00D4
:104B40000A00121212160A000A0E111F111111008A
:104B50000A0E111111110E000A11111111110E007E
:104B60000C12121C12121C100000000000000000A9
:104B7000000000000000000000183C3C3C18180039
:104B8000181800000066666624000000000000009F
:104B900000000000006C6CFE6C6C6CFE6C6C000025
:104BA0000018187CC6C2C07C0686C67C1818000097
:104BB000000000C2C60C183066C6000000000038B5
:104BC0006C6C3876DCCCCC760000001818183000FD
:104BD00000000000000000000000000C1830303021
:104BE0003030180C000000000030180C0C0C0C0CBD
:104BF000183000000000000000663CFF3C6600002A
:104C00000000000000000018187E181800000000C6
:104C1000000000000000000000181818300000001C
:104C20000000000000FE0000000000000000000086
:104C30000000000000001818000000000002060C30
:104C4000183060C080000000000000386CC6C6D676
:104C5000C6C66C38000000000018387818181818FC
:104C6000187E00000000007CC6060C183060C6FEEE
:104C700000000000007CC606063C0606C67C00005C
:104C80000000000C1C3C6CCCFE0C0C1E0000000054
:104C900000FEC0C0C0FC0606C67C00000000003854
:104CA00060C0C0FCC6C6C67C0000000000FEC60690
:104CB0000C183030303000000000007CC6C6C67CC6
:104CC000C6C6C67C00000000007CC6C6C67E0606BE
:104CD0000C780000000000001818000000181800F0
:104CE0000000000000001818000000181830000034
:104CF0000000000C183060C06030180C000000008C
:104D0000000000007E00007E000000000000006047
:104D100030180C060C18306000000000007CC6C67D
:104D20000C181800181800000000007CC6C6DEDE53
:104D3000DEDCC07C000000000010386CC6C6FEC679
:104D4000C6C60000000000FC6666667C666666FCFF
:104D500000000000003C66C2C0C0C0C2663C00004B
:104D6000000000F86C66666666666CF8000000007D
:104D700000FE66626878686266FE0000000000FE61
:104D800066626878686060F000000000003C66C2FF
:104D9000C0C0DEC6663A0000000000C6C6C6C6FE39
:104DA000C6C6C6C600000000003C1818181818181F
:104DB000183C00000000001E0C0C0C0C0CCCCC7835
:104DC0000000000000E6666C6C786C6C66E6000023
:104DD000000000F060606060606266FE000000003D
:104DE00000C6EEFED6C6C6C6C6C60000000000C697
:104DF000E6F6FEDECEC6C6C600000000007CC6C6D3
:104E0000C6C6C6C6C67C0000000000FC6666667C9E
:104E1000606060F000000000007CC6C6C6C6C6D652
:104E2000DE7C0E00000000FC6666667C6C6666E652
:104E300000000000007CC6C660380CC6C67C0000BE
:104E40000000007E7E5A18181818183C0000000058
:104E500000C6C6C6C6C6C6C6C67C0000000000C6E0
:104E6000C6C6C6C6C66C38100000000000C6C6C65E
:104E7000C6D6D6FE6C6C0000000000C6C6C67C38E4
:104E80007CC6C6C60000000000666666663C181850
:104E9000183C0000000000FEC68C183060C2C6FE40
:104EA00000000000003C303030303030303C00003A
:104EB00000000080C0E070381C0E060200000000F8
:104EC000003C0C0C0C0C0C0C0C3C000010386CC69C
:104ED00000000000000000000000000000000000D2
:104EE00000000000000000FF0030180C000000006F
:104EF000000000000000000000000000780C7CCCE6
:104F0000CC760000000000E06060786C6666667C2D
:104F100000000000000000007CC6C0C0C67C00008D
:104F20000000001C0C0C3C6CCCCCCC7600000000CB
:104F3000000000007CC6FEC0C67C00000000001C13
:104F40003632307C30303078000000000000000045
:104F500076CCCCCC7C0CCC78000000E060606C7629
:104F6000666666E600000000001818003818181879
:104F7000183C00000000000606000E060606066645
:104F8000663C000000E06060666C786C66E60000DD
:104F900000000038181818181818183C00000000F5
:104FA00000000000ECFED6D6D6D6000000000000BF
:104FB0000000DC6666666666000000000000000017
:104FC0007CC6C6C6C67C0000000000000000DC668F
:104FD00066667C6060F000000000000076CCCCCCFF
:104FE0007C0C0C1E000000000000DC76666060F0A7
:104FF00000000000000000007CC6701CC67C0000A1
:10500000000000103030FC303030361C0000000052
:1050100000000000CCCCCCCCCC760000000000001E
:105020000000C6C6C66C381000000000000000007A
:10503000C6C6D6D6FE6C0000000000000000C66C9C
:1050400038386CC60000000000000000C6C6C6C6A6
:105050007E060C78000000000000FECC183066FED2
:1050600000000000000E181818701818180E000024
:105070000000001818181818181818180000000058
:1050800000701818180E181818700000FF000000A3
:10509000000000000000000000FF000000480000C9
:1050A000780C7CCCCC7600000000004800007CC668
:1050B000C6C6C67C0000000000480000CCCCCCCCAA
:1050C000CC76000000440010386CC6C6FEC6C6C6CA
:1050D00000000044007CC6C6C6C6C6C6C67C00002A
:1050E000004400C6C6C6C6C6C6C6C67C00000000D0
:1050F0000078CCCCF8CCCCCCF8C0C0C08E2E9F2E83
:105100008BB7809300010895E82DF92D809100015F
:105110008BBF88940895481A8827580A0895480E26
:105120008827581E0895ED91FC91EF5FFF4FFC9387
:10513000EE930895ED91FC91E150F040FC93EE93D5
:10514000089509D00E946D2A00FC10D0089503D064
:105150001ED001F8F9CF0024E89457FF02C009D00F
:10516000689400F80BD010F80124089502D009D0FB
:105170000895509540954F5F5F4F0895E89417FF4D
:105180000895009510950F5F1F4F68940895352F6F
:10519000242FE894452B11F468940895512F402F43
:1051A0000027112780E1440F551F001F111F021B0C
:1051B000130B416018F4020F131F4E7F8A9599F765
:1051C00008958F938D918823E9F711978F91089512
:1051D000A0E8BFE017D08D3049F0883079F0332354
:1051E000C9F38D933A9563FE31D0F4CF63FC03C0CD
:1051F0002DD08AE02BD088278C93089527D0119743
:105200003395E8CF7F930F929F93AF93BF93809195
:105210002B018823E1F3F89480912B018A958093E8
:105220002B0190912901A1E0B1E0A90F0024B01D4C
:105230008C919395983209F4992790932901789449
:10524000BF91AF919F910F907F9108959F939FB7CA
:105250009F93AF93BF930F937F9390915601983292
:10526000E1F3F89490915601939590935601992704
:1052700000915501ACE2B1E0A00FB91F8C930395EA
:10528000083209F400270093550180919A0080624A
:1052900080939A007F910F91BF91AF919F919FBF93
:1052A0009F9108953197F1F708950E9466298D9195
:1052B0000E9468299A95D9F70E9467290895B99A9A
:1052C000BB98C39ABA9A80E58DB908950895089558
:1052D0008FB9779BFECF8FB10895689462F80895D7
:1052E000E89462F80895EF93FF93EE27E82BE92BFB
:1052F00031F0E0EAFFE03197F1F70197D1F7FF9144
:10530000EF9108955A924A92480E8827581E0895A0
:105310008DE207FD8D938F2D881F802F881F8F575B
:10532000082F6894F7F8802F87FF15C08095839524
:10533000082F80E38D938EE28D93802F815228F089
:1053400080E38D9399279C93089544270A95802F95
:1053500009F198D01FC0805230F09EE49D9381E403
:105360008D939D93EFCF4427DF92EF92FF920F939F
:105370008FE1801B11F0082F85D08BD09EE29D938A
:105380000F91FF90EF90DF9044270395003209F4CE
:10539000D7CF2DD03F93E4E2F4E50E94462D38E1CB
:1053A0002F2D1E2D0D2DFF24EE24DD244427000F6C
:1053B000111F221FA8F42F923F920E94E42B102C61
:1053C0000E94E42B202C0E94E42B302C0E94E42B22
:1053D0003197410DD21CE31CF01C3F902F9001C06F
:1053E000339631963A9519F73F9107D0ADCFDD0C42
:1053F000EE1CFF1C0A95D9F70895002719E058D034
:105400008F93802B11F0039501C08F911A95B9F7F6
:10541000802F882309F494CF8F91805D8D930A9516
:10542000D9F790CF0065CD1D80B2E60E40597307C5
:10543000A0ACB90350D6DC01286BEE0094357700A0
:10544000CA9A3B0065CD1D00B2E60E0059730700F5
:10545000ACB90300D6DC01006BEE0000357700002C
:105460009A3B0000CD1D0000E60E0000730700000F
:10547000B9030000DC010000EE000000770000002E
:105480003B000000F694E794D79447950A95D1F72E
:10549000089500270DD08F9303958F2D8E298D2988
:1054A000842BC1F78F91805D8D930A95D9F74ACFF0
:1054B0001F930F93002710E2440FDD1CEE1CFF1C0E
:1054C000001F802F9AE0890B10F0082F43951A9542
:1054D00099F7802F0F911F9108950F92B801469F61
:1054E0008001479F100D569F100D0F9008950E9448
:1054F000E42B0D920020D9F70895903051F000244C
:105500000D911C91000F111F001D9A95D9F71C9346
:105510000E930895903051F00D911C9116950795BA
:1055200008F410689A95D1F71C930E930895903063
:1055300029F08C91880F9A95E9F78C930895903013
:1055400041F00D911C91000F111F9A95E1F71C93EA
:105550000E930895903041F00D911C91169507958A
:105560009A95E1F71C930E93089599910027A90F3E
:10557000B01F1197492F4A95FBB65E2F6F2FE89405
:1055800011274395203019F0D895802D01C08081D6
:105590008823E1F07C917723C9F0781759F40EF055
:1055A000042F139568941196319658F78BB783950D
:1055B0008BBFE7CF112321F0411BA11B1127B10B9A
:1055C000E894E52FF62FFBBE1196DBCF882311F070
:1055D00000270895089533D0992711278F2D880F1C
:1055E00080E8F82A802F881F08F41FEF41F08F57BA
:1055F000082F07FD04C0003240F08FEF01C088275C
:10560000982FD82EE82EF82E09C08FE1801B082F86
:10561000F694E794D79497950A95D1F7112351F012
:105620009095D094E094F09481E0980F8827D81E4C
:10563000E81EF81E0F2DFE2CED2CD92E0895D190CA
:10564000E190F19001910895219131914191519111
:105650000895102F90E8FF0C001F0927990FF79469
:105660001078652F90E8440F551F5927990F4795DB
:10567000607800380895FF0C90E89027110F9795F7
:10568000F794092F0895502F2D2D3E2D4F2D612F6A
:1056900008952DEC3CEC4CEC5DE366270FC0CFDFAA
:1056A000F2DFDD24EE2490E8F92E0FE307C0CCDF13
:1056B00005C02227332740E251E46627552351F1E4
:1056C000002381F1C6DF71F1162700585058089465
:1056D000050B18F407FD03C025C007FD23C0469540
:1056E00037952795F694E794D79422D0FF202AF097
:1056F000DD0CEE1CFF1C015073F09D2D969548F0BB
:10570000DD203AF4EE202AF491E0D90E9927E91E23
:10571000F91EB1CF07C09FE7092FF92A9FEFD92EB5
:10572000E92E0895DD24EE24FF2400271127089593
:105730009F929924AA24BB2488E1D216E306F4069A
:1057400028F0D21AE30AF40A089401C08894991C3C
:10575000AA1CBB1CDD0CEE1CFF1C8A9571F7D92C12
:10576000EA2CFB2C9F90089574DFE1F25038D1F2BF
:105770001627005850580894051F12F418F4CBCF80
:1057800008F0D0CF0AD0FF202AF0BB0CDD1CEE1CA5
:10579000FF1C71CF0F5FFBF16ECF9F929924AA245B
:1057A000BB24992788E1990CAA1CBB1CDD1CEE1CAC
:1057B000FF1C30F4920EA31EB41ED91EE91EF91E62
:1057C0008A9589F79F900895D895319628F48F93FC
:1057D0008BB783958BBF8F9100200895F5DF202D27
:1057E000F3DF302DF1DF402DEFDF502D089507FB63
:1057F00000680EF40F7757FB50680EF45F7707FDD3
:1058000002C057FF05C0D216E306F4060507089547
:105810002D153E054F05500708950E947029E89404
:1058200088278A938A937EDF11278D918032E9F34E
:105830001197BBD098F08D3229F4109511968C9168
:10584000B4D060F08E3229F411968C91AED008F469
:1058500046C022960E946D2981E008958C91A5D0C2
:10586000D8F547D01196D0F703958D919ED0E0F3EF
:105870008E3229F48C9199D010F41196FBCF853497
:1058800019F0853609F055C011968C918ED060F0D4
:105890008D3219F08B3221F0DCCF08800094088221
:1058A00011968C9182D0A8F68053898311968C91A1
:1058B0007CD058F49981990F990F0980900D990F18
:1058C0008053890F8983873220F6898198819923B3
:1058D0000AF48195080F2DC08E3289F611968C91AD
:1058E00064D068F606D018F011960A95F8CF119694
:1058F000C1CF4F2D3E2D2D2DDD0CEE1CFF1CA8F031
:10590000DD0CEE1CFF1C88F0D20EE31EF41E68F0C6
:10591000DD0CEE1CFF1C48F0805309F06894D80E93
:105920008827E81EF81E08F00895F42EE32ED22EE4
:10593000089534D019F116F5098308E921D00695A8
:10594000882787959F2D9F77980FF92E0150000F7C
:10595000110F07958981882379F01AF4819589833D
:1059600006C097DE89818A958983D9F705C0A1DEB3
:1059700089818A958983D9F722960895D3DEFCCF51
:105980000DD041F0FF2032F00A9531F0DD0CEE1C15
:10599000FF1CD2F7889408950894089500240D28D8
:1059A0000E280F28002A00200895803320F08A3323
:1059B00010F4089408958894089591E005C092E049
:1059C00003C094E001C098E028F48F938BB78395CF
:1059D0008BBF8F91F9DE0D929A95E1F70895E80F4C
:1059E000F91FEBCF91E0882321F08894991F8A95C5
:1059F000E9F7892F90950895883018F0119688500E
:105A0000FBCF08952E2E3F2E992781918D3209F0DC
:105A100093958823D1F79A95E22DF32D112361F008
:105A2000091718F011F0101B01C0191B28F021F004
:105A300080E28D931A95E9F780818D3219F48D9368
:105A4000319604C0222311F08BE28D93091738F0B0
:105A500031F0091B21F080E38D930A95E9F78191DC
:105A60008D938823E1F7332351F0EA2FFB2F3196F2
:105A700033958E9182933A95E1F78EE28C93089557
:105A80000F9301E00BBF0F91889408950F930027A7
:105A9000F9CF0F9302E0F6CF0F9303E0F3CF7F939C
:105AA0000F93AF93BF938F939F938FB78F93E89488
:105AB00080912B0108E2081B29F490919C000E9420
:105AC0006D2914C000912A01A1E0B1E077279091DF
:105AD0009C00A00FB71F9C936894839580932B0123
:105AE0000395083209F4002700932A019D3011F430
:105AF0000E9410018F918FBF9F918F91BF91AF91A5
:105B00000F917F9118957F93AF93BF938F939F933E
:105B10008FB78F93909156019923A1F09A95909306
:105B200056019927ACE2B1E080915401A80FB91F4A
:105B30009C918395883209F488278093540190932F
:105B40009C0005C080919A008F7D80939A008F9170
:105B50008FBF9F918F91BF91AF917F9118956FB734
:105B6000F894882793E08D939A95E9F76FBF08958D
:105B7000040F151F261F371F0895000F111F221F26
:105B8000331F089500951095209530950F5F1F4F96
:105B90002F4F3F4F0895019110810EC00191119137
:105BA000219130810BC00191108117FF05C03FEF9B
:105BB0002FEF04C0008111272227332737FF03C0AE
:105BC000E1DF8DE28D93CF93DF93CF92DF92EF925F
:105BD000AA24BB24CC24DD24EE2440E2CAE0DD2745
:105BE00055E093E38881890F87FD9F7083FD907F47
:105BF000891B89935A95A9F7C0DFAA1CBB1CCC1C32
:105C0000DD1CEE1C4A9551F7E894EFE0FF278291E6
:105C10000ED0EB30E0F71EF068948A2D0CD0882768
:105C20008D93EF90DF90CF90DF91CF910895982FD3
:105C3000829501D0892F8F70805D26F0803309F422
:105C4000089568948D9308950027112722273327FC
:105C50001DD08A3328F4803318F005D015D0F9CF41
:105C60000EF490CF089580538F93402F512F622FC1
:105C7000732F83DF82DF7CDF80DF8F919927080F0E
:105C8000191F291F391F08958D910895E894FCDF8D
:105C90008032E9F38B32D9F38930C9F38D3211F4B4
:105CA0006894F2CF089588278D93089581918D93FC
:105CB0008823E1F7089594E081918D939A95E1F717
:105CC000089509919191992351F08A95D9F73197C7
:105CD00081918D930A9519F08823D1F70895E3CF28
:105CE0008FEF83959D919923E1F70895689401C002
:105CF000E894AF93BF938D9116F0919103C00E94E9
:105D0000E42B902D891718F011F48823A1F7BF9187
:105D1000AF910895E89463F80895689463F808953E
:105D200000000000000080BF0000A04000002043F1
:105D3000000020410000304100004041000050417F
:105D4000000060414B59063D0000C0410000C841C1
:105D50000000E8413A002A003D00202020202020B9
:105D60002020202020202020202020202020000073
:105D70005374F672756E6721204144584C206C6F45
:105D800077005374F672756E6721204144584C2099
:105D90006869676800005374F672756E6721204762
:105DA00079726F206C6F77005374F672756E67218D
:105DB000204779726F206869676800005374F67233
:105DC000756E6721204675DF736368616C74657258
:105DD00000005374616E646279005600206B6D2F71
:025DE000680059
:00000001FF
